:020000040000FA
:04080000A6EF06F069
:1008100003B207EF05F0F2B422EF05F09EB02AEF25
:1008200005F09EB232EF05F0F2A81AEF04F0F2B232
:100830001CEF04F084EF06F0CD90F2929EA026EF1C
:1008400004F00101533F26EF04F0542BAEC1B2F186
:10085000AFC1B3F1B0C1B4F1B1C1B5F1AAC1AEF14C
:10086000ABC1AFF1ACC1B0F1ADC1B1F1A6C1AAF15C
:10087000A7C1ABF1A8C1ACF1A9C1ADF1A2C1A6F16C
:10088000A3C1A7F1A4C1A8F1A5C1A9F19EC1A2F17C
:100890009FC1A3F1A0C1A4F1A1C1A5F19AC19EF18C
:1008A0009BC19FF19CC1A0F19DC1A1F196C19AF19C
:1008B00097C19BF198C19CF199C19DF1CECF96F162
:1008C000CFCF97F153C198F154C199F1CF6ACE6A55
:1008D0000101536B546B9E90CD800EBC0E8E0EBAF0
:1008E00075EF04F00E8A84EF06F00E8C0EBEB1EFA9
:1008F00004F096C19AF197C19BF198C19CF199C1FE
:100900009DF19AC19EF19BC19FF19CC1A0F19DC137
:10091000A1F19EC1A2F19FC1A3F1A0C1A4F1A1C107
:10092000A5F1A2C1A6F1A3C1A7F1A4C1A8F1A5C1D7
:10093000A9F1A6C1AAF1A7C1ABF1A8C1ACF1A9C1A7
:10094000ADF1AAC1AEF1ABC1AFF1ACC1B0F1ADC177
:10095000B1F1AEC1B2F1AFC1B3F1B0C1B4F1B1C147
:10096000B5F101015E6B5F6B606B616B96515E2749
:1009700097515F2398516023995161239A515E27C3
:100980009B515F239C5160239D5161239E515E27A3
:100990009F515F23A0516023A1516123A2515E2783
:1009A000A3515F23A4516023A5516123A6515E2763
:1009B000A7515F23A8516023A9516123AA515E2743
:1009C000AB515F23AC516023AD516123AE515E2723
:1009D000AF515F23B0516023B1516123B2515E2703
:1009E000B3515F23B4516023B5516123D890613373
:1009F00060335F335E33D890613360335F335E338F
:100A0000D890613360335F335E3384EF06F0039236
:100A1000030103EE00F080517F0BE92604C0EFFFD5
:100A2000802B8151805D700BD8A48B820000805197
:100A3000815D700BD8A48B9281518019D8B4079036
:100A400084EF06F0F2940101453F84EF06F0462B57
:100A500084EF06F09E900101533F84EF06F0542B83
:100A600084EF06F09E92C3CF55F1C4CF56F1C282F7
:100A700007B49DEF05F047C14BF148C14CF149C1A6
:100A80004DF14AC14EF15EC162F15FC163F160C1D7
:100A900064F161C165F196C1B6F197C1B7F198C132
:100AA000B8F199C1B9F19AC1BAF19BC1BBF19CC12E
:100AB000BCF19DC1BDF19EC1BEF19FC1BFF1A0C1FE
:100AC000C0F1A1C1C1F1A2C1C2F1A3C1C3F1A4C1CE
:100AD000C4F1A5C1C5F1A6C1C6F1A7C1C7F1A8C19E
:100AE000C8F1A9C1C9F1AAC1CAF1ABC1CBF1ACC16E
:100AF000CCF1ADC1CDF1AEC1CEF1AFC1CFF1B0C13E
:100B0000D0F1B1C1D1F1B2C1D2F1B3C1D3F1B4C10D
:100B1000D4F1B5C1D5F1010155515B2756515C2384
:100B2000E86A5D230D2E9DEF05F05CC157F15DC1B4
:100B300058F15B6B5C6B5D6B078E0201002F84EFDD
:100B400006F03C0E006F00C10CF101C10DF102C1B5
:100B50000EF103C10FF104C110F105C111F106C17D
:100B600012F107C113F108C114F109C115F10AC14D
:100B700016F10BC117F134C135F101018A67C8EFD5
:100B800005F08B67C8EF05F08C67C8EF05F08D673F
:100B9000CCEF05F0FCEF05F08EC100F18FC101F143
:100BA00090C102F191C103F10101010E046F000E29
:100BB000056F000E066F000E076F25EC14F000C1E4
:100BC0008EF101C18FF102C190F103C191F1006773
:100BD000F1EF05F00167F1EF05F00267F1EF05F0C5
:100BE0000367FCEF05F08AC18EF18BC18FF18CC1D8
:100BF00090F18DC191F10E80D57ED5BE69D0D6CF52
:100C000047F1D7CF48F145C149F1E86AE8CF4AF149
:100C10000F9047C100F148C101F149C102F14AC139
:100C200003F101010A0E046F000E056F000E066F3E
:100C3000000E076F25EC14F000AF0F80010154A7E0
:100C40002EEF06F00E9A0E9C0E9E0101000E5E6FB6
:100C5000600E5F6F3D0E606F080E616F010147BF50
:100C60003EEF06F048673EEF06F049673EEF06F0BC
:100C70004A673EEF06F0F28863EF06F0F2985E6B8B
:100C80005F6B606B616B966B976B986B996B9A6BF4
:100C90009B6B9C6B9D6B9E6B9F6BA06BA16BA26B08
:100CA000A36BA46BA56BA66BA76BA86BA96BAA6BB8
:100CB000AB6BAC6BAD6BAE6BAF6BB06BB16BB26B68
:100CC000B36BB46BB56BD76AD66A0101456B466BE3
:100CD0000CC100F10DC101F10EC102F10FC103F110
:100CE00010C104F111C105F112C106F113C107F1E0
:100CF00014C108F115C109F116C10AF117C10BF1B0
:100D000035C134F184EF06F002C0E0FF005001C0AD
:100D1000D8FF1000A6B28AEF06F00CC0A9FF0BC0E6
:100D2000A8FFA69EA69CA684F29E550EA76EAA0EAC
:100D3000A76EA682F28EA694A6B29CEF06F01200D1
:100D4000A96EA69EA69CA680A8501200076A0E6AED
:100D50000F6A0F010E0EC16E860EC06E030EC26EBC
:100D60000F01896A110E926E080E8A6EF10E936E53
:100D70008B6A800E946EF18E0D6A01015B6B5C6B69
:100D80005D6B576B586BF29A0101476B486B496B6F
:100D90004A6B4B6B4C6B4D6B4E6B4F6B506B516B8F
:100DA000526B456B466BD76AD66A0F01280ED56E1B
:100DB000F28A9D90B00ECD6E01015E6B5F6B606B31
:100DC000616B626B636B646B656B666B676B686BA7
:100DD000696B536B546BCF6ACE6A0E9A0E9C0E9E53
:100DE0009D80760ECA6E9D8202013C0E006FCC6A19
:100DF000160EA0EC06F0E8CF00F1170EA0EC06F0FE
:100E0000E8CF01F1180EA0EC06F0E8CF02F1190EC0
:100E1000A0EC06F0E8CF03F1010103AF2AEF07F0E1
:100E20001CEC15F0160E0C6E00C10BF08AEC06F0EF
:100E3000170E0C6E01C10BF08AEC06F0180E0C6E4A
:100E400002C10BF08AEC06F0190E0C6E03C10BF018
:100E50008AEC06F000C18AF101C18BF102C18CF16C
:100E600003C18DF100C18EF101C18FF102C190F17A
:100E700003C191F11A0EA0EC06F0E8CF00F11B0EB1
:100E8000A0EC06F0E8CF01F11C0EA0EC06F0E8CFD4
:100E900002F11D0EA0EC06F0E8CF03F1010103AF53
:100EA00080EF07F01CEC15F01A0E0C6E00C10BF071
:100EB0008AEC06F01B0E0C6E01C10BF08AEC06F0FA
:100EC0001C0E0C6E02C10BF08AEC06F01D0E0C6EAF
:100ED00003C10BF08AEC06F01A0EA0EC06F0E8CF86
:100EE00000F11B0EA0EC06F0E8CF01F11C0EA0EC07
:100EF00006F0E8CF02F11D0EA0EC06F0E8CF03F1FA
:100F000000C192F101C193F102C194F103C195F1C5
:100F1000240EAC6E900EAB6E240EAC6E080EB86E46
:100F2000000EB06E1F0EAF6E0401806B816B0F015F
:100F3000900EAB6E0F019D8A0301806B816BA26BDB
:100F40008B9207900001F28EF28C07B0E9EF11F05E
:100F50000EB0CAEF0CF00301805181197F0BD8B499
:100F6000E9EF11F013EE00F081517F0BE126812BA8
:100F7000E7CFE8FFE00BD8B4E9EF11F023EE82F001
:100F8000A2511F0BD926E7CFDFFFA22BDF50780A33
:100F9000D8A4E9EF11F007808EC100F18FC101F1F3
:100FA00090C102F191C103F10101040E046F000E22
:100FB000056F000E066F000E076F25EC14F000AFF2
:100FC000EBEF07F00101030E8E6F000E8F6F000E26
:100FD000906F000E916F03018251720AD8B4CAEF6C
:100FE0000CF08251520AD8B4CAEF0CF08251750A43
:100FF000D8B4CAEF0CF08251630AD8B4A5EF0EF052
:101000008251690AD8B485EF09F082517A0AD8B4BE
:1010100098EF0AF08251490AD8B424EF09F08251BE
:10102000500AD8B442EF08F08251700AD8B485EF64
:1010300008F08251540AD8B4B0EF08F08251740A13
:10104000D8B4F6EF08F08251730AD8B4FAEF0BF077
:101050008251530AD8B45FEF0CF0DAEF0EF00401BE
:1010600014EE00F080517F0BE12682C4E7FF802B55
:1010700012000D0E826F2FEC08F00A0E826F2FEC1B
:1010800008F0120083C32AF184C32BF185C32CF12D
:1010900086C32DF187C32EF188C32FF189C330F1A8
:1010A0008AC331F18BC332F18CC333F101016AEC95
:1010B00015F0E1EC14F0160E0C6E00C10BF08AEC8A
:1010C00006F0170E0C6E01C10BF08AEC06F0180E3C
:1010D0000C6E02C10BF08AEC06F0190E0C6E03C107
:1010E0000BF08AEC06F000C18AF101C18BF102C15C
:1010F0008CF103C18DF100C18EF101C18FF102C1EC
:1011000090F103C191F124EF09F083C32AF184C364
:101110002BF185C32CF186C32DF187C32EF188C333
:101120002FF189C330F18AC331F18BC332F18CC303
:1011300033F101016AEC15F0E1EC14F000C18AF121
:1011400001C18BF102C18CF103C18DF100C18EF19F
:1011500001C18FF102C190F103C191F124EF09F0B7
:1011600083C32AF184C32BF185C32CF186C32DF1EF
:1011700087C32EF188C32FF189C330F18AC331F1BF
:101180008CC332F18DC333F101016AEC15F0E1EC4F
:1011900014F00101000E046F000E056F010E066FC2
:1011A000000E076F34EC14F01A0E0C6E00C10BF039
:1011B0008AEC06F01B0E0C6E01C10BF08AEC06F0F7
:1011C0001C0E0C6E02C10BF08AEC06F01D0E0C6EAC
:1011D00003C10BF08AEC06F000C192F101C193F15A
:1011E00002C194F103C195F124EF09F083C32AF100
:1011F00084C32BF185C32CF186C32DF187C32EF157
:1012000088C32FF189C330F18AC331F18CC332F125
:101210008DC333F101016AEC15F0E1EC14F001012A
:10122000000E046F000E056F010E066F000E076FB3
:1012300034EC14F000C192F101C193F102C194F1B8
:1012400003C195F124EF09F0160EA0EC06F0E8CFEB
:1012500000F1170EA0EC06F0E8CF01F1180EA0EC9B
:1012600006F0E8CF02F1190EA0EC06F0E8CF03F18A
:10127000BFEC14F0EBEC12F00401730E826F2FEC54
:1012800008F004012C0E826F2FEC08F08AC100F1E7
:101290008BC101F18CC102F18DC103F1BFEC14F0DF
:1012A000EBEC12F00401730E826F2FEC08F00401D6
:1012B0002C0E826F2FEC08F01A0EA0EC06F0E8CF8F
:1012C00000F11B0EA0EC06F0E8CF01F11C0EA0EC23
:1012D00006F0E8CF02F11D0EA0EC06F0E8CF03F116
:1012E000F5EC0EF004012C0E826F2FEC08F092C189
:1012F00000F193C101F194C102F195C103F1F5EC44
:101300000EF039EC08F0DAEF0EF00401690E826F8E
:101310002FEC08F004012C0E826F2FEC08F0010175
:10132000040E006F000E016F000E026F000E036FBF
:10133000BFEC14F02CC182F40401300E82272FEC94
:1013400008F02DC182F40401300E82272FEC08F042
:101350002EC182F40401300E82272FEC08F02FC139
:1013600082F40401300E82272FEC08F030C182F4A1
:101370000401300E82272FEC08F031C182F4040101
:10138000300E82272FEC08F032C182F40401300EB7
:1013900082272FEC08F033C182F40401300E82273B
:1013A0002FEC08F004012C0E826F2FEC08F00101E5
:1013B000030E006F000E016F000E026F000E036F30
:1013C000BFEC14F02CC182F40401300E82272FEC04
:1013D00008F02DC182F40401300E82272FEC08F0B2
:1013E0002EC182F40401300E82272FEC08F02FC1A9
:1013F00082F40401300E82272FEC08F030C182F411
:101400000401300E82272FEC08F031C182F4040170
:10141000300E82272FEC08F032C182F40401300E26
:1014200082272FEC08F033C182F40401300E8227AA
:101430002FEC08F004012C0E826F2FEC08F0010154
:10144000190E006F000E016F000E026F000E036F89
:10145000BFEC14F02CC182F40401300E82272FEC73
:1014600008F02DC182F40401300E82272FEC08F021
:101470002EC182F40401300E82272FEC08F02FC118
:1014800082F40401300E82272FEC08F030C182F480
:101490000401300E82272FEC08F031C182F40401E0
:1014A000300E82272FEC08F032C182F40401300E96
:1014B00082272FEC08F033C182F40401300E82271A
:1014C0002FEC08F004012C0E826F2FEC08F0200E98
:1014D000F86EF76AF66A04010900F5CF82F42FEC82
:1014E00008F00900F5CF82F42FEC08F00900F5CFE1
:1014F00082F42FEC08F00900F5CF82F42FEC08F00D
:101500000900F5CF82F42FEC08F00900F5CF82F442
:101510002FEC08F00900F5CF82F42FEC08F0090059
:10152000F5CF82F42FEC08F039EC08F0DAEF0EF08A
:101530008351630AD8A4DAEF0EF08451610AD8A46B
:10154000DAEF0EF085516C0AD8A4DAEF0EF086516E
:10155000410A42E08651440A1BE08651420AD8B44F
:10156000FFEF0AF08651350AD8B464EF10F08651C7
:10157000360AD8B4B9EF10F08651370AD8B422EF42
:1015800011F08651380AD8B480EF11F0DAEF0EF07E
:101590000798079A04017A0E826F2FEC08F0040175
:1015A000780E826F2FEC08F00401640E826F2FEC2E
:1015B00008F081A8E3EF0AF00401550E826F2FECCA
:1015C00008F0E8EF0AF004014C0E826F2FEC08F0EF
:1015D00039EC08F0DAEF0EF00788079A04017A0E6A
:1015E000826F2FEC08F00401410E826F2FEC08F09F
:1015F0000401610E826F2FEC08F0D9EF0AF0079812
:10160000078A04017A0E826F2FEC08F00401420E63
:10161000826F2FEC08F00401610E826F2FEC08F04E
:10162000D9EF0AF0010166671DEF0BF067671DEF48
:101630000BF068671DEF0BF0696735EF0BF04F6734
:1016400029EF0BF0506729EF0BF0516729EF0BF0F2
:10165000526735EF0BF00101000E006F000E016FB5
:10166000000E026F000E036F12000101620E046F84
:10167000010E056F000E066F000E076F66C100F1C8
:1016800067C101F168C102F169C103F125EC14F0F1
:1016900003BFB9EF0BF00101000E046FA80E056F38
:1016A000550E066F020E076F66C100F167C101F1AA
:1016B00068C102F169C103F166C186F167C187F1B2
:1016C00068C188F169C189F125EC14F003BF72EF9C
:1016D0000BF00101000E866FA80E876F550E886F04
:1016E000020E896F0E0EA0EC06F0E8CF18F10F0E77
:1016F000A0EC06F0E8CF19F1100EA0EC06F0E8CF50
:101700001AF1110EA0EC06F0E8CF1BF16EEC13F00D
:1017100086C104F187C105F188C106F189C107F1CD
:1017200025EC14F0078232EC13F06EEC13F0079204
:1017300032EC13F086C100F187C101F188C102F1DA
:1017400089C103F1079232EC13F0CC0E046FE00E66
:10175000056F870E066F050E076F25EC14F000C1AC
:1017600018F101C119F102C11AF103C11BF1F1EF26
:101770000BF00101800E006F1A0E016F060E026F52
:10178000000E036F4FC104F150C105F151C106F1C4
:1017900052C107F125EC14F003AFD2EF0BF01CECB3
:1017A00015F012000E0EA0EC06F0E8CF18F10F0EA7
:1017B000A0EC06F0E8CF19F1100EA0EC06F0E8CF8F
:1017C0001AF1110EA0EC06F0E8CF1BF14FC100F1A9
:1017D00050C101F151C102F152C103F1078232EC53
:1017E00013F018C100F119C101F11AC102F11BC1B6
:1017F00003F112000401730E826F2FEC08F0040154
:101800002C0E826F2FEC08F0078462C166F163C171
:1018100067F164C168F165C169F14BC14FF14CC119
:1018200050F14DC151F14EC152F157C159F158C15A
:101830005AF1079420EC0CF039EC08F0DAEF0EF0D6
:1018400066C100F167C101F168C102F169C103F12C
:101850000101BFEC14F0EBEC12F00401630E826F97
:101860002FEC08F004012C0E826F2FEC08F04FC112
:1018700000F150C101F151C102F152C103F1010166
:10188000BFEC14F0EBEC12F00401660E826F2FEC4B
:1018900008F004012C0E826F2FEC08F01CEC15F000
:1018A00059C100F15AC101F10101BFEC14F0EBEC98
:1018B00012F00401740E826F2FEC08F012000F82F8
:1018C0000401530E826F2FEC08F004012C0E826F7E
:1018D0002FEC08F083C32AF184C32BF185C32CF1CC
:1018E00086C32DF187C32EF188C32FF189C330F150
:1018F0008AC331F18BC332F18CC333F101016AEC3D
:1019000015F0E1EC14F000C166F101C167F102C10C
:1019100068F103C169F18EC32AF18FC32BF190C323
:101920002CF191C32DF192C32EF193C32FF194C3E7
:1019300030F195C331F196C332F197C333F1010110
:101940006AEC15F0E1EC14F000C14FF101C150F167
:1019500002C151F103C152F15DEC15F099C32FF1B1
:101960009AC330F19BC331F19CC332F19DC333F173
:1019700001016AEC15F0E1EC14F000C159F101C16C
:101980005AF120EC0CF004012C0E826F2FEC08F0C1
:10199000D1EF0CF08251520A03E10E82D1EF0CF02C
:1019A0000E928251750A03E10F84D8EF0CF00F9468
:1019B0008251550A03E10F86DFEF0CF00F96078482
:1019C0000FB23CEF0DF00FA428EF0DF0B6C166F199
:1019D000B7C167F1B8C168F1B9C169F1BAC16AF1BB
:1019E000BBC16BF1BCC16CF1BDC16DF1BEC16EF18B
:1019F000BFC16FF1C0C170F1C1C171F1C2C172F15B
:101A0000C3C173F1C4C174F1C5C175F1C6C176F12A
:101A1000C7C177F1C8C178F1C9C179F1CAC17AF1FA
:101A2000CBC17BF1CCC17CF1CDC17DF1CEC17EF1CA
:101A3000CFC17FF1D0C180F1D1C181F1D2C182F19A
:101A4000D3C183F1D4C184F1D5C185F130EF0DF05C
:101A500062C166F163C167F164C168F165C169F192
:101A60004BC14FF14CC150F14DC151F14EC152F13A
:101A700057C159F158C15AF107940EA05EEF0DF00D
:101A8000010192674BEF0DF093674BEF0DF09467F8
:101A90004BEF0DF095674FEF0DF05EEF0DF012EC90
:101AA0000BF092C104F193C105F194C106F195C107
:101AB00007F125EC14F003BFA2EF0EF012EC0BF0CF
:101AC0000101000E046F000E056F010E066F000E7F
:101AD000076F53EC14F00FA475EF0DF00401750EB1
:101AE000826F2FEC08F07AEF0DF00401720E826F16
:101AF0002FEC08F004012C0E826F2FEC08F0BFECE5
:101B000014F0296789EF0DF00401200E826F8CEF2D
:101B10000DF004012D0E826F2FEC08F030C182F41D
:101B20000401300E82272FEC08F031C182F4040149
:101B3000300E82272FEC08F004012E0E826F2FEC5E
:101B400008F032C182F40401300E82272FEC08F035
:101B500033C182F40401300E82272FEC08F0040117
:101B60006D0E826F2FEC08F004012C0E826F2FECAB
:101B700008F04FC100F150C101F151C102F152C151
:101B800003F10101BFEC14F0EBEC12F00401480E7C
:101B9000826F2FEC08F004017A0E826F2FEC08F0B0
:101BA00004012C0E826F2FEC08F066C100F167C1B2
:101BB00001F168C102F169C103F10101BFEC14F048
:101BC000EBEC12F00401630E826F2FEC08F00401BD
:101BD0002C0E826F2FEC08F066C100F167C101F195
:101BE00068C102F169C103F101010A0E046F000E20
:101BF000056F000E066F000E076F34EC14F0000E38
:101C0000046F120E056F000E066F000E076F53EC87
:101C100014F0BFEC14F02AC182F40401300E8227C4
:101C20002FEC08F02BC182F40401300E82272FEC38
:101C300008F02CC182F40401300E82272FEC08F04A
:101C40002DC182F40401300E82272FEC08F02EC142
:101C500082F40401300E82272FEC08F02FC182F4A9
:101C60000401300E82272FEC08F030C182F4040109
:101C7000300E82272FEC08F004012E0E826F2FEC1D
:101C800008F031C182F40401300E82272FEC08F0F5
:101C900032C182F40401300E82272FEC08F033C1E8
:101CA00082F40401300E82272FEC08F00401730E39
:101CB000826F2FEC08F004012C0E826F2FEC08F0DD
:101CC0001CEC15F059C100F15AC101F104EC10F0FF
:101CD0000EB26EEF0EF00EA0A0EF0EF004012C0E6F
:101CE000826F2FEC08F0200EF86EF76AF66A040196
:101CF0000900F5CF82F42FEC08F00900F5CF82F44B
:101D00002FEC08F00900F5CF82F42FEC08F0090061
:101D1000F5CF82F42FEC08F00900F5CF82F42FEC18
:101D200008F00900F5CF82F42FEC08F00900F5CF98
:101D300082F42FEC08F00900F5CF82F42FEC08F0C4
:101D400039EC08F00E90DAEF0EF00401630E826FAA
:101D50002FEC08F004012C0E826F2FEC08F0E0EC61
:101D60000EF004012C0E826F2FEC08F053EC0FF0F4
:101D700004012C0E826F2FEC08F0CFEC0FF0040161
:101D80002C0E826F2FEC08F00101F80E006FCD0EC3
:101D9000016F660E026F030E036FF5EC0EF0040187
:101DA0002C0E826F2FEC08F0E5EC0FF039EC08F008
:101DB000DAEF0EF00301A26B07900F92E9EF11F03A
:101DC000D8900E0EA0EC06F0E8CF00F10F0EA0ECBC
:101DD00006F0E8CF01F1100EA0EC06F0E8CF02F11A
:101DE000110EA0EC06F0E8CF03F10101000E046F24
:101DF000000E056F010E066F000E076F53EC14F016
:101E0000BFEC14F02AC182F40401300E82272FECBB
:101E100008F02BC182F40401300E82272FEC08F069
:101E20002CC182F40401300E82272FEC08F02DC162
:101E300082F40401300E82272FEC08F02EC182F4C8
:101E40000401300E82272FEC08F02FC182F4040128
:101E5000300E82272FEC08F030C182F40401300EDE
:101E600082272FEC08F031C182F40401300E822762
:101E70002FEC08F004012E0E826F2FEC08F032C117
:101E800082F40401300E82272FEC08F033C182F473
:101E90000401300E82272FEC08F004016D0E826FD2
:101EA0002FEC08F01200120EA0EC06F0E8CF00F1C3
:101EB000130EA0EC06F0E8CF01F1140EA0EC06F032
:101EC000E8CF02F1150EA0EC06F0E8CF03F1010116
:101ED0000A0E046F000E056F000E066F000E076FEE
:101EE00034EC14F0000E046F120E056F000E066F36
:101EF000000E076F53EC14F0BFEC14F02AC182F40B
:101F00000401300E82272FEC08F02BC182F404016B
:101F1000300E82272FEC08F02CC182F40401300E21
:101F200082272FEC08F02DC182F40401300E8227A5
:101F30002FEC08F02EC182F40401300E82272FEC22
:101F400008F02FC182F40401300E82272FEC08F034
:101F500030C182F40401300E82272FEC08F0040116
:101F60002E0E826F2FEC08F031C182F40401300E86
:101F700082272FEC08F032C182F40401300E822750
:101F80002FEC08F033C182F40401300E82272FECCD
:101F900008F00401730E826F2FEC08F012000A0E95
:101FA000A0EC06F0E8CF00F10B0EA0EC06F0E8CFB5
:101FB00001F10C0EA0EC06F0E8CF02F10D0EA0EC42
:101FC00006F0E8CF03F104EF10F0060EA0EC06F0E7
:101FD000E8CF00F1070EA0EC06F0E8CF01F1080E03
:101FE000A0EC06F0E8CF02F1090EA0EC06F0E8CF75
:101FF00003F104EF10F001011CEC15F0078457C148
:1020000000F158C101F107940101E80E046F800E40
:10201000056F000E066F000E076F34EC14F0000E13
:10202000046F040E056F000E066F000E076F53EC71
:1020300014F0880E046F130E056F000E066F000E6D
:10204000076F25EC14F00A0E046F000E056F000EEA
:10205000066F000E076F53EC14F0BFEC14F0010193
:10206000296738EF10F00401200E826F3BEF10F06B
:1020700004012D0E826F2FEC08F030C182F40401B0
:10208000300E82272FEC08F031C182F40401300EAB
:1020900082272FEC08F032C182F40401300E82272F
:1020A0002FEC08F004012E0E826F2FEC08F033C1E4
:1020B00082F40401300E82272FEC08F00401430E55
:1020C000826F2FEC08F0120087C32AF188C32BF12E
:1020D00089C32CF18AC32DF18BC32EF18CC32FF150
:1020E0008DC330F18EC331F190C332F191C333F11E
:1020F0000101296B6AEC15F0E1EC14F00101000E0E
:10210000046F000E056F010E066F000E076F34ECB2
:1021100014F00E0E0C6E00C10BF08AEC06F00F0EE0
:102120000C6E01C10BF08AEC06F0100E0C6E02C1B1
:102130000BF08AEC06F0110E0C6E03C10BF08AEC6A
:1021400006F004017A0E826F2FEC08F004012C0EC9
:10215000826F2FEC08F00401350E826F2FEC08F02F
:1021600004012C0E826F2FEC08F0E0EC0EF0E8EF8B
:102170000AF087C32AF188C32BF189C32CF18AC3E3
:102180002DF18BC32EF18CC32FF18DC330F18EC393
:1021900031F190C332F191C333F10101296B6AEC43
:1021A00015F0E1EC14F0880E046F130E056F000EAD
:1021B000066F000E076F29EC14F0000E046F040E7A
:1021C000056F000E066F000E076F34EC14F001016E
:1021D000E80E046F800E056F000E066F000E076F8D
:1021E00053EC14F00A0E0C6E00C10BF08AEC06F0F2
:1021F0000B0E0C6E01C10BF08AEC06F00C0E0C6E8F
:1022000002C10BF08AEC06F00D0E0C6E03C10BF050
:102210008AEC06F004017A0E826F2FEC08F00401BC
:102220002C0E826F2FEC08F00401360E826F2FEC1B
:1022300008F004012C0E826F2FEC08F0CFEC0FF0A9
:10224000E8EF0AF087C32AF188C32BF189C32CF188
:102250008AC32DF18BC32EF18CC32FF18DC330F1C6
:102260008FC331F190C332F191C333F101016AECB4
:1022700015F0E1EC14F0000E046F120E056F000E65
:10228000066F000E076F34EC14F001010A0E046FA4
:10229000000E056F000E066F000E076F53EC14F072
:1022A000120E0C6E00C10BF08AEC06F0130E0C6ED1
:1022B00001C10BF08AEC06F0140E0C6E02C10BF09B
:1022C0008AEC06F0150E0C6E03C10BF08AEC06F0DA
:1022D00004017A0E826F2FEC08F004012C0E826F3D
:1022E0002FEC08F00401370E826F2FEC08F0040188
:1022F0002C0E826F2FEC08F053EC0FF0E8EF0AF091
:1023000087C32AF188C32BF189C32CF18AC32DF12D
:102310008BC32EF18CC32FF18DC330F18EC331F1FD
:1023200090C332F191C333F10101296B6AEC15F0CE
:10233000E1EC14F0880E046F130E056F000E066FAB
:10234000000E076F29EC14F0000E046F040E056FE9
:10235000000E066F000E076F34EC14F00101E80E5A
:10236000046F800E056F000E066F000E076F53ECB2
:1023700014F0060E0C6E00C10BF08AEC06F0070E8E
:102380000C6E01C10BF08AEC06F0080E0C6E02C157
:102390000BF08AEC06F0090E0C6E03C10BF08AEC10
:1023A00006F004017A0E826F2FEC08F004012C0E67
:1023B000826F2FEC08F00401380E826F2FEC08F0CA
:1023C00004012C0E826F2FEC08F0E5EC0FF0E8EF23
:1023D0000AF081A8A7EF12F007A860EF12F0010140
:1023E000800E006F1A0E016F060E026F000E036F53
:1023F0004BC104F14CC105F14DC106F14EC107F1CD
:1024000025EC14F003BFA7EF12F0E5EC12F04BC17E
:1024100000F14CC101F14DC102F14EC103F107823F
:1024200032EC13F018C104F119C105F11AC106F11B
:102430001BC107F1F80E006FCD0E016F660E026F23
:10244000030E036F25EC14F00E0E0C6E00C10BF0A2
:102450008AEC06F00F0E0C6E01C10BF08AEC06F050
:10246000100E0C6E02C10BF08AEC06F0110E0C6E11
:1024700003C10BF08AEC06F0078401011CEC15F097
:1024800057C100F158C101F107940A0E0C6E00C14A
:102490000BF08AEC06F00B0E0C6E01C10BF08AEC0F
:1024A00006F00C0E0C6E02C10BF08AEC06F00D0E5D
:1024B0000C6E03C10BF08AEC06F00798A7EF12F040
:1024C00007AAA7EF12F0078401011CEC15F057C111
:1024D00000F158C101F10794060E0C6E00C10BF01B
:1024E0008AEC06F0070E0C6E01C10BF08AEC06F0C8
:1024F000080E0C6E02C10BF08AEC06F0090E0C6E91
:1025000003C10BF08AEC06F0078462C100F163C1DD
:1025100001F164C102F165C103F10794120E0C6E62
:1025200000C10BF08AEC06F0130E0C6E01C10BF02B
:102530008AEC06F0140E0C6E02C10BF08AEC06F069
:10254000150E0C6E03C10BF08AEC06F0079A04011D
:10255000805181197F0B0BE09EA809D014EE00F08A
:1025600081517F0BE126E750812B0F01AD6EA5EF66
:1025700007F018C100F119C101F11AC102F11BC124
:1025800003F1000E046F000E056F010E066F000EC2
:10259000076F53EC14F029A1E4EF12F02051D8B4E6
:1025A000E4EF12F018C100F119C101F11AC102F1F2
:1025B0001BC103F1000E046F000E056F0A0E066FBB
:1025C000000E076F53EC14F012000101186B196B29
:1025D0001A6B1B6B12002AC182F40401300E822791
:1025E0002FEC08F02BC182F40401300E82272FEC6F
:1025F00008F02CC182F40401300E82272FEC08F081
:102600002DC182F40401300E82272FEC08F02EC178
:1026100082F40401300E82272FEC08F02FC182F4DF
:102620000401300E82272FEC08F030C182F404013F
:10263000300E82272FEC08F031C182F40401300EF5
:1026400082272FEC08F032C182F40401300E822779
:102650002FEC08F033C182F40401300E82272FECF6
:1026600008F012000101005305E1015303E1025398
:1026700001E1002BF5EC13F01CEC15F03951006F63
:102680003A51016F420E046F4B0E056F000E066F3C
:10269000000E076F34EC14F000C104F101C105F124
:1026A00002C106F103C107F118C100F119C101F11E
:1026B0001AC102F11BC103F107B263EF13F029EC59
:1026C00014F065EF13F025EC14F000C118F101C10E
:1026D00019F102C11AF103C11BF112001CEC15F033
:1026E00059C100F15AC101F1060EA0EC06F0E8CF85
:1026F00004F1070EA0EC06F0E8CF05F1080EA0ECFF
:1027000006F0E8CF06F1090EA0EC06F0E8CF07F1DD
:1027100025EC14F000C124F101C125F102C126F11C
:1027200003C127F1290E046F000E056F000E066F1E
:10273000000E076F34EC14F0EE0E046F430E056FBD
:10274000000E066F000E076F29EC14F024C104F18F
:1027500025C105F126C106F127C107F134EC14F0BB
:1027600000C11CF101C11DF102C11EF103C11FF125
:10277000120EA0EC06F0E8CF04F1130EA0EC06F068
:10278000E8CF05F1140EA0EC06F0E8CF06F1150E27
:10279000A0EC06F0E8CF07F10D0E006F000E016F00
:1027A000000E026F000E036F34EC14F0180E046F6D
:1027B000000E056F000E066F000E076F53EC14F04D
:1027C0001CC104F11DC105F11EC106F11FC107F1B5
:1027D00029EC14F06A0E046F2A0E056F000E066FC6
:1027E000000E076F25EC14F01200BF0EFA6E200EDB
:1027F0003A6F396BD8900037013702370337D8B0BA
:1028000006EF14F03A2FFBEF13F039073A070353A2
:10281000D8B412000331070B80093F6F03390F0B47
:10282000010F396F80EC5FF0406F390580EC5FF08D
:10283000405D405F396B3F33D8B0392739333FA90A
:102840001BEF14F040513927120041EC15F0D8B0BD
:10285000120003510719346F04EC15F0D89007519A
:10286000031934AF800F1200346B28EC15F0D8A098
:102870003EEC15F0D8B0120013EC15F01CEC15F07E
:102880001F0E366F54EC15F00B35D8B004EC15F074
:10289000D8A00335D8B01200362F42EF14F034B16F
:1028A0002BEC15F01200346B0451051106110711C1
:1028B0000008D8A028EC15F0D8A03EEC15F0D8B050
:1028C0001200086B096B0A6B0B6B54EC15F01F0EB2
:1028D000366F54EC15F007510B5DD8A47CEF14F063
:1028E00006510A5DD8A47CEF14F00551095DD8A407
:1028F0007CEF14F00451085DD8A08FEF14F0045160
:10290000085F0551D8A0053D095F0651D8A0063DD6
:102910000A5F0751D8A0073D0B5FD8900081362F82
:1029200069EF14F034B12BEC15F0346B28EC15F092
:10293000D89058EC15F007510B5DD8A4ACEF14F00B
:1029400006510A5DD8A4ACEF14F00551095DD8A476
:10295000ACEF14F00451085DD8A0BBEF14F0003FB9
:10296000BBEF14F0013FBBEF14F0023FBBEF14F0DC
:10297000032BD8B4120034B12BEC15F01200010176
:10298000346B28EC15F0D8B012005DEC15F0200E79
:10299000366F003701370237033711EE33F00A0E76
:1029A000376FE7360A0EE75CD8B0E76EE552372F8F
:1029B000D1EF14F0362FC9EF14F034B12981D8903B
:1029C000120001010A0E346F200E366F11EE29F04D
:1029D0003451376F0A0ED890E652D8B0E726E73266
:1029E000372FECEF14F00333023301330033362F6B
:1029F000E6EF14F0E750FF0FD8A00335D8B012006F
:102A000029B12BEC15F01200045100270551D8B064
:102A1000053D01270651D8B0063D02270751D8B021
:102A2000073D032712000051086F0151096F025141
:102A30000A6F03510B6F12000101006B016B026BF7
:102A4000036B12000101046B056B066B076B120030
:102A50000335D8A012000351800B001F011F021F75
:102A6000031F003F3BEF15F0013F3BEF15F0023F26
:102A70003BEF15F0032B342B032512000735D8A0AC
:102A800012000751800B041F051F061F071F043F7C
:102A900051EF15F0053F51EF15F0063F51EF15F0DE
:102AA000072B342B07251200003701370237033775
:102AB000083709370A370B3712000101296B2A6BD7
:102AC0002B6B2C6B2D6B2E6B2F6B306B316B326B3A
:102AD000336B12002A510F0B2A6F2B510F0B2B6FE8
:102AE0002C510F0B2C6F2D510F0B2D6F2E510F0BE7
:102AF0002E6F2F510F0B2F6F30510F0B306F315145
:102B00000F0B316F32510F0B326F33510F0B336F8D
:022B10001200B1
:10BF0000E844F926000C160C2B0C3F0C520C640C68
:10BF1000760C860C960CA50CB30CC10CCF0CDC0C6B
:06BF2000E80CF40C000C1B
:00000001FF
